S02200006F70656E626C745F6E75636C656F5F73746D33326631303372622E7372656343
S3150800000010080020C51B0008151C0008191C00084C
S315080000101D1C0008211C0008251C00080000000003
S31508000020000000000000000000000000291C000875
S315080000302D1C000800000000311C0008C90C00082F
S31508000040351C0008391C00083D1C0008411C000826
S31508000050451C0008491C00084D1C0008511C0008D6
S31508000060551C0008591C00085D1C0008611C000886
S31508000070651C0008691C00086D1C0008711C000836
S31508000080751C0008791C00087D1C0008811C0008E6
S31508000090851C0008891C00088D1C0008911C000896
S315080000A0951C0008991C00089D1C0008A11C000846
S315080000B0A51C0008A91C0008AD1C0008B11C0008F6
S315080000C0B51C0008B91C0008BD1C0008C11C0008A6
S315080000D0C51C0008C91C0008CD1C0008D11C000856
S315080000E0D51C0008D91C0008DD1C00080020DFF814
S315080000F0681408700020DFF8601488640020DFF8B0
S31508000100581481F843000020DFF84C14A1F8440085
S315080001100020DFF8441488700020DFF83C1448708B
S315080001207047DFF834040078002801D1002000E089
S31508000130012070470020DFF8201481F8430070473B
S3150800014080B50178FF291ED100F095F8DFF808047C
S3150800015090F84300012802D1102000F082F8DFF859
S31508000160F803B0F9440001280CDB0120DFF8E81396
S3150800017081F84300DFF8E003B0F94410DFF8DC0348
S3150800018000F053F801BDDFF8D013097801294BD1E7
S315080001900178C92932D0CC293FD0CF293AD0D029E5
S315080001A02FD0D12933D0D2292ED0F32917D0F4292C
S315080001B00FD0F5290AD0F6290ED0FA2912D0FC2933
S315080001C013D0FD2914D0FE2915D029E000F0D5F862
S315080001D0BCE700F0F5F8B9E700F0C4F8B6E700F0B8
S315080001E015F9B3E700F0A6F8B0E700F09EF8ADE71A
S315080001F000F083F8AAE700F072F8A7E700F039F9EB
S31508000200A4E700F058F9A1E700F017F99EE700F017
S3150800021084F99BE700F095F998E700F0A7F995E7C8
S31508000220202000F01EF891E7ACE780B589B200F00F
S31508000230BDF901BDF8B504000D001600002704E05D
S315080002402078C719641C00F0F9F92800451E002813
S31508000250F6D1FFB237600120F2BD0020BE494870D2
S315080002607047FE21BC4AD170BB4908710220BA49C1
S31508000270A1F84400704780B5FFF7EFFF0120B649A3
S315080002800870FF20B449C8700020B3490871B24805
S31508000290007950F01000B04908710020AE49487145
S315080002A0AD484079AC49487100F08BF9AA49887184
S315080002B000F09CF9A849C87100F098F980B2000AC4
S315080002C0A54908720120A44948720120A2498872EA
S315080002D00820A149A1F8440000F0B4F901BD80B591
S315080002E000209D490870FFF7B8FFFF209A49C8709B
S315080002F001209949A1F8440001BDFF209649C8701C
S31508000300002095490871944840789349487100201F
S315080003109149887100209049C87100208E49087259
S3150800032006208D49A1F84400704780B50020FFF7E4
S3150800033098FF01BDFF208849C870894886498864A6
S3150800034000208549087100208349487100208249A8
S31508000350887107208049C1F8070008207E49A1F85E
S3150800036044007047FF217C4AD17040687A49886406
S3150800037001207949A1F84400704710B5040000F03F
S3150800038020F980B2401E6178884203DA2220FFF7FE
S3150800039068FF14E06278734892B26F49896C00F07E
S315080003A095F9FF206C49C8706B48806C617808180D
S315080003B0694988646078401C6749A1F8440010BD03
S315080003C010B5040000F0FDF880B2401E617888423E
S315080003D003DA2220FFF745FF17E060685E49886464
S315080003E06278604892B25C49896C00F06FF9FF2028
S315080003F05949C8705848806C617808185649886405
S315080004006078401C5449A1F8440010BD80B5FF210E
S31508000410514AD170544A41684F48806CFFF70AFF29
S315080004204D49087100204C49487100204A49887195
S3150800043008204949A1F8440001BD80B5FF20464976
S31508000440C87000204449087100204349487100F0EB
S31508000450B8F84149887100203F49C87100203E49D3
S31508000460087200203C49487207203B49A1F844001D
S3150800047001BD10B5040000F0A4F8621C80B2411E4C
S315080004803548806C00F0E2F8002803D13120FFF7E8
S31508000490E8FE0FE0FF203049C87000F092F82E49B8
S315080004A0896C80B2401E40182B49886401202A496D
S315080004B0A1F8440010BD10B5040000F082F880B21F
S315080004C0801E6178884203DA2220FFF7CAFE23E0FD
S315080004D0FF202149C87001201F49A1F8440060780F
S315080004E0002807D100F0C2F8002802D13120FFF712
S315080004F0B8FE11E0A21C61781748806C00F0A6F8D7
S31508000500002803D13120FFF7ACFE05E01248806CC5
S31508000510617808181049886410BD80B541680E488E
S31508000520806C00F097F8002803D13120FFF799FE78
S3150800053006E0FF200849C87001200749A1F84400D1
S3150800054001BD80B500F0A0F8FF200349C87001205E
S315080005500149A1F8440001BD180C00201B0C00201D
S315080005600C1C00081C0C00201F0C002080B5312034
S31508000570FFF777FE01BD000080B5FFF7B7FD00F075
S31508000580D5F800202449087001BD80B5694623487E
S3150800059000F006F9012807D100201F4908709DF8C8
S315080005A000101E48FFF7CCFD01BD704780B51A4AFA
S315080005B01278002A02D1C9B200F0D3F8FFF7BAFDC3
S315080005C001BD15480078002805D0022807D004D3B5
S315080005D0032806D007E0402006E0002004E00020BB
S315080005E002E0002000E0402080B270470A48007808
S315080005F0002805D0022807D004D3032806D007E030
S31508000600402006E0002004E0002002E0002000E090
S31508000610402080B27047000008000020A80C002087
S3150800062010B50024FFF77DFD002800D00124200026
S31508000630C0B210BD80B500F053F901BD80B500F019
S3150800064054F901BD80B500F055F901BD80B500F03B
S315080006505AF902BD80B500F086F902BD80B500F0F2
S315080006600BFA02BD80B500F050FA02BD80B500F065
S31508000670C8F9002801D1002001E000F02BFA02BDDC
S3150800068080B500F0EAFA01BD10B5FFF7E7FF0028CC
S3150800069016D000F014F9002812D0FFF786FF00F0F4
S315080006A0F1FA00F024FBFFF7DDFF0649084006498A
S315080006B00860FFF7D7FF001D046800F0D0FAA047CE
S315080006C010BD000080FFFF1F08ED00E070B50400B4
S315080006D00D00160005E0287820706D1C641CFFF7D5
S315080006E0ADFF3000461E80B20028F4D170BD000070
S315080006F0C16851F40051C1607047016931F49041F5
S315080007000161416931F02A01416170470068400979
S3150800071010F0010070470068C00910F0010070472A
S315080007204068C0B27047C9B24160704700B587B02B
S315080007304FF46140009000200190002002900020B4
S3150800074003900C2004900020059069464E4800F05E
S315080007503AFB4D48FFF7D1FF4B48FFF7C9FF07B0F3
S3150800076000BD70B504000D00EDB2412D03DB6F210D
S31508000770464800F06FFB2800C0B200F06EF800266D
S3150800078006E0FFF75BFFB6B2A05D00F066F8761CE0
S3150800079030002900C9B280B289B28842F1D370BD4F
S315080007A038B504000D003A480078002817D13948B2
S315080007B000F044F801283FD13648007800283BD09D
S315080007C034480078412837DA00F06AFA3249086076
S315080007D000203249087001202D4908702CE02D4868
S315080007E02E4909780844401C00F028F8012819D138
S315080007F02A480078401C2949087028480078254965
S315080008000978884218D12548027892B224492000EE
S31508000810FFF75CFF00201E49087020480078287002
S3150800082001200AE000F03CFA1B490968643181425C
S3150800083002D2002016490870002032BD10B5040007
S315080008401148FFF763FF002805D00F48FFF768FF38
S315080008502070012000E0002010BD10B50100C9B2CB
S315080008600948FFF760FF00F01BFA10F10A04064872
S31508000870FFF751FF002805D1FFF7E0FE00F010FA58
S315080008808442F4D210BD000000440040881A0008D3
S31508000890210D0020640C0020180D0020200D0020DA
S315080008A0650C0020806810EA112080B2C1F30F2180
S315080008B0884201D1012000E00020C0B2704780B50F
S315080008C005490648FFF7EEFF002801D1002002E09F
S315080008D000F0F3FA012002BD2000200400100140B8
S315080008E080B5642000F0C2FA01BD80B500F0C1FAF7
S315080008F001BD00005FF0FF309F4908605FF0FF30E0
S315080009009E490860704710B50B009D49096F9C4CBD
S31508000910646F6118491E091A5C1EA14201D20020A3
S3150800092020E097490968884209D39549096F944C8C
S31508000930646F6118491E1C18641EA14201D200206A
S3150800094010E0410A4FF4007461438D4C2468A142BB
S3150800095004D10100894800F015F903E00100864832
S3150800096000F010F910BD70B586B00022009201247F
S31508000970834A126F824B5B6F9A18521E121A4B1ECD
S315080009809A4201D200203AE0820A4FF480635A4321
S315080009907B4B1B689A4209D3794B1B6F784D6D6F59
S315080009A0EB185B1E0D186D1EAB4201D2002026E027
S315080009B04018801A850A800500D06D1C0020019019
S315080009C003920120049000F0E1FA002604E003985F
S315080009D010F580600390761C3000290080B289B239
S315080009E0884208D2FFF72AFE694601A800F066FB8E
S315080009F00028ECD0002400F0DBFA2000C0B206B0D4
S31508000A0070BD80B5002000905C48006810F1010FA9
S31508000A1001D101202FE0009858494968081800902C
S31508000A200098564989680818009000985349C9687B
S31508000A30081800900098514909690818009000980C
S31508000A404E4949690818009000984C498969081860
S31508000A50009000984949C969081800900098C04351
S31508000A6000900098401C00906A460421444800689B
S31508000A70EC30FFF748FF02BD0020414909680968C4
S31508000A8008183F490968091D096808183C49096892
S31508000A900831096808183A4909680C3109680818BC
S31508000AA03749096810310968081835490968143141
S31508000AB00968081832490968183109680818304958
S31508000AC00968EC3109680818002801D1012000E0FE
S31508000AD00020704780B52948006810F1010F06D03C
S31508000AE0264800F092F8002801D100200CE02248A0
S31508000AF0006810F1010F06D01F4800F086F800289C
S31508000B0001D1002000E0012002BD1D4800687047A1
S31508000B1080B5CA0501D000200BE002688A4201D1DF
S31508000B20012006E001604FF40072001DFFF7CEFDBC
S31508000B30012002BD38B504000D001048844208D1D2
S31508000B400D4C29002000FFF7E3FF002810D10020F4
S31508000B500FE00B480068854203D1084C0848056831
S31508000B60EFE7200000F051F80028EAD1002000E065
S31508000B70200032BD0000000010080020140A0020E2
S31508000B80541900082DE9F04104000F0015001E0055
S31508000B90780A4FF4007101FB00F8206810F1010F84
S31508000BA007D141462000FFF7B3FF002801D10020F6
S31508000BB029E02068404508D041462000FFF7BAFFE3
S31508000BC00400002C01D100201DE02068381A2044BA
S31508000BD0071DFFF733FD201D381AB0F5007F0AD32D
S31508000BE018F500712000FFF7A5FF0400002C01D1BD
S31508000BF0002008E0271D287838707F1C6D1C761E9B
S31508000C00002EE6D10120BDE8F0812DE9F04105006E
S31508000C10012600F0BBF9002700E07F1C802F16D2C2
S31508000C20286810EB870805EB87004468FFF706FD80
S31508000C30220000234146022000F04EF9002801D088
S31508000C40002604E0D8F80000A042E6D0002600F00E
S31508000C50AFF93000C0B2BDE8F08172B6704762B62F
S31508000C607047000080B500F00DF81048104908607C
S31508000C7000201049086005200F49086000200F4928
S31508000C80086001BD00200C49086070470A480068E2
S31508000C90C00304D509480068401C08490860704725
S31508000CA080B5FFF7F3FF0548006802BD3F1901004C
S31508000CB014E000E018E000E010E000E0140D002069
S31508000CC080B5FFF7EDFF02BD7047000080B51148FB
S31508000CD0006850F010000F490860032000F0CCFAB5
S31508000CE0002000F0F1FA00F0E2FB002002BD80B51A
S31508000CF05FF0FF30084908600020084908605FF087
S31508000D00FF300549086000200349086000F014FC1C
S31508000D10002002BD002002400C10024010100240C4
S31508000D20C068400B10F001007047026932F4405267
S31508000D30114301617047426932F4407211434161BF
S31508000D40704770B4192303FB01F39400B3FBF4F363
S31508000D506424B3FBF4F3192404FB01F49500B4FBF3
S31508000D60F5F4192505FB01F59600B5FBF6F564269D
S31508000D70B5FBF6F5642606FB1544240132346425D2
S31508000D80B4FBF5F414F0F00414EB0313192404FB74
S31508000D9001F49500B4FBF5F4192569439200B1FBFB
S31508000DA0F2F16422B1FBF2F1642202FB114109015E
S31508000DB032316422B1FBF2F111F00F01C91889B280
S31508000DC0816070BC7047F0B585B004000D00002640
S31508000DD000272000FFF7A4FF00282DD1E0681C4952
S31508000DE0084069680843E968084329690843E060D8
S31508000DF0A9682000FFF799FF69692000FFF79BFFA4
S31508000E00684600F0EAFB0F48844201D1039F08E0D8
S31508000E100D48844201D1029F03E00C48844200D168
S31508000E20029F002F08D02868002805D001262A68C6
S31508000E3039002000FFF785FF3000C0B205B0F0BDCD
S31508000E40000000000038014000440040004800400F
S31508000E50F3E9FFFF80B5FFF7F1FBFCE7C1F30F21CC
S31508000E6001617047C1F30F21416170471649088037
S31508000E70704780B5FFF714FF1449096888421BD3E9
S31508000E8013480078002808D101201149087042F259
S31508000E9020011048FFF7E2FF07E000200C49087020
S31508000EA042F220010B48FFF7DDFFFFF7F9FE06497E
S31508000EB0098808180549086001BD80B542F2200175
S31508000EC00448FFF7CFFF01BD1C0D0020100D0020C0
S31508000ED01F0D0020000801402DE9F84381460E0049
S31508000EE014001D0001205FF000080027DFF8B0019C
S31508000EF0007E012801D1022046E00120DFF8A0117A
S31508000F0008764CF2503000F066F8C0B2002836D1A8
S31508000F10B9F1010F01D1012705E0B9F1020F01D19D
S31508000F20022700E004275FF0000801E018F1010835
S31508000F3041463A00C9B2D2B2914220D220002900D5
S31508000F405FFA88F85FEA081200F0B2FB02000B00AD
S31508000F50110089B25FFA88F816EB480000F030F8FD
S31508000F604CF2503000F037F8DFF8381109684908B4
S31508000F704900DFF830211160C0B20028D6D0002120
S31508000F80DFF81C211176C0B2BDE8F283002045497E
S31508000F90096809060AD54549454A11604549444A3A
S31508000FA0116040490968090600D50120C0B270479A
S31508000FB03C48006850F080003A49086000207047B5
S31508000FC00022374BDA61374A126852F00102354B74
S31508000FD01A600180704738B50400FFF771FE0500F6
S31508000FE031480068C0070BD514F1010FF8D0002C62
S31508000FF004D0FFF765FE401B8442F1D2032017E0B8
S3150800100029480068800602D5202027490860264816
S315080010100068C00607D428480068C00703D42248D9
S315080010200068400703D500F004F8012000E000201E
S3150800103032BD00201C490968C90607D51849C9697F
S3150800104051F00201164AD16150F01000164909689C
S31508001050490707D51249C96951F00101104AD161FA
S3150800106050F0040014490968C9070BD50C49C96929
S3150800107051F004010A4AD1610F4909684908490033
S315080010800D4A116040F20111884206D10A480068EB
S31508001090400840000849086001E0034908607047B5
S315080010A0E80C0020102002400C200240230167456E
S315080010B004200240AB89EFCD1C200240F8B504009D
S315080010C00D0001260027DFF8F000007E012801D177
S315080010D002204CE00120DFF8E0100876206802289C
S315080010E016D14CF25030FFF776FF002839D101208F
S315080010F000F03EF84CF25030FFF76DFF0600DFF8BF
S31508001100BC00006830F00400DFF8B010086028E082
S315080011104CF25030FFF75FFF002822D15FF0FF3016
S315080011202860A76801E017F58067E0684FF48061DA
S31508001130A26801FB0020874213D2380000F029F884
S315080011404CF25030FFF747FF0600DFF870000068E2
S3150800115030F00200DFF864100860F6B2002EE2D024
S315080011602F600020DFF8501008763000C0B2F2BDBC
S315080011700020DFF84410C8611048006850F00400E9
S315080011800E4908600D48006850F040000B49086099
S3150800119070470021084AD1610849096851F00201DF
S315080011A0064A1160064908600448006850F0400085
S315080011B00249086070470000E80C00201020024031
S315080011C01420024010F00701384800684FF6FF0265
S315080011D01040374A52EA01210843344908607047EB
S315080011E032480068C0F30220704740B2002808D58C
S315080011F00901304A40B210F00F00104400F8041CF0
S3150800120003E009012C4A40B21154704710B410F09B
S315080012100700D0F10703052B01D3042301E0D0F121
S315080012200703041D072C01D2002000E0C01E01247C
S3150800123014FA03F35B1E19408140012313FA00F0E8
S31508001240401E1040084310BC704780B5411EB1F1DE
S31508001250807F01D301200EE0401E184908600F2147
S315080012605FF0FF30FFF7C1FF00201549086007202F
S3150800127014490860002002BD80B5FFF7A3FF01BD31
S3150800128070B504000D0016000020FFF7A9FF320014
S315080012902900FFF7BBFF0100200040B2FFF7A5FFBA
S315080012A070BD80B5FFF7D1FF02BD00000CED00E070
S315080012B00000FA0518ED00E000E400E014E000E0A4
S315080012C018E000E010E000E010B504004FF47A7072
S315080012D00D490978B0FBF1F00C490968B1FBF0F04B
S315080012E0FFF7DFFF002801D001200CE0102C09D2FF
S315080012F0002221005FF0FF30FFF7C2FF04480460B8
S31508001300002000E0012010BD090000200400002094
S31508001310000000209548006850F480209349086032
S3150800132070479248006850F48030904908607047CA
S315080013308E480068400C10F0010070478C49096817
S315080013408908890008438A49086070478848006800
S3150800135010F00C0070478649096831F0F00108431F
S315080013608349086070478249096831F4E061084397
S315080013707F49086070477E49096831F4605108431F
S315080013807B49086070477948006850F08070774953
S315080013900860704775480068400E10F001007047F5
S315080013A0734A126832F47C1210F440301043084332
S315080013B06F490860704781B06E49096801436D4AF4
S315080013C011606C49096808400090009801B07047A0
S315080013D06849096831EA000066490860704781B0C3
S315080013E0654909680143644A116063490968084008
S315080013F00090009801B070475F49096831EA00001B
S315080014005D49086070475D490968C908C90008430D
S315080014105A49086070475948006810F00700704735
S31508001420C1F30F214161704780B500F005F800F05F
S315080014304EF900F05AF9FCE780B5FFF747FC00F0D3
S3150800144001F801BD80B50220FFF7DDFFFFF7E3FFD6
S31508001450022803D065214A48FFF7FCFCFFF75AFF2C
S31508001460FFF75FFFFFF764FF0128FBD15FF4E01188
S315080014705FF48030FFF794FFFFF785FFFFF78AFFD9
S315080014800128FBD10020FFF766FF4FF48060FFF7C5
S315080014906AFF0020FFF76FFF0220FFF74FFFFFF7F5
S315080014A055FF0828FBD1374800F02AF901BD00B5D9
S315080014B085B00120FFF793FF5FF08050FFF77BFFB1
S315080014C00420FFF78CFF1020FFF789FF5FF4003038
S315080014D0FFF771FF42F220000090012001900220E0
S315080014E00290002003906946274800F0BFF942F2AF
S315080014F020012548FFF794FF244800900420019016
S315080015006946234800F0B2F940F2044000900920E9
S315080015100190022002900020039069461A4800F0C4
S31508001520A5F940F60800009009200190694616487A
S3150800153000F09CF905B000BD80B5154800F051F9DA
S31508001540114800F04EF95FF40030FFF741FF102014
S31508001550FFF752FF0420FFF74FFF5FF08050FFF7B9
S3150800156037FF0120FFF748FF01BD000000100240C9
S31508001570041002401C1002401810024000200240CD
S31508001580341A000800A24A0400080140200020047A
S31508001590001001404148006810F00C0070473F48B1
S315080015A0006810F0F00070473C48006810F4E060EE
S315080015B070473A48006810F460507047374800682A
S315080015C010F4803070473548006810F47010704782
S315080015D03248006810F40030704710B5040000F077
S315080015E00EF82060206800F01EF86060606800F061
S315080015F025F8A060606800F02BF8E06010BD80B5A3
S315080016000020FFF7C7FF002804D0042804D00828C4
S3150800161004D006E0224805E0214803E000F022F85D
S3150800162000E01F4802BD10B50400FFF7B8FF1D49CA
S31508001630C0F30310085CC440200010BD10B50400B8
S31508001640FFF7B2FF1849000A085CC440200010BD25
S3150800165010B50400FFF7ADFF1349C00A085CC44083
S31508001660200010BD10B500240020FFF7A7FF0028B2
S3150800167003D0B0F5803F02D008E00C4C07E0FFF736
S31508001680A7FF401C0649B1FBF0F400E0074CFFF742
S315080016909AFF800C801C00FB04F010BD0410024069
S315080016A000127A00DC1B0008041C000800093D0033
S315080016B0D2B2203A22BF21FA02F000217047203226
S315080016C0D141D04048409140D1404840704780B50C
S315080016D0FEF7D6FFFEF7AEFFFFF7C4FAFEF7B2FF36
S315080016E0FEF74AFF00F002F901BD80B5FEF7A6FF36
S315080016F0FFF7CCFAFEF749FF00F001F901BD00003B
S3150800170001490860704700000400002030B410EB5F
S31508001710116091FAA1F3B3FA83F391FAA1F1B1FA40
S3150800172081F104680F25DBB29B0015FA03F334EA4E
S315080017300303C9B2890012FA01F11943016030BCEA
S31508001740704730B410EB116091FAA1F3B3FA83F342
S3150800175091FAA1F1B1FA81F104680325DBB29B0085
S3150800176015FA03F334EA0303C9B2890012FA01F140
S315080017701943016030BC704730B410EB116091FA20
S31508001780A1F3B3FA83F391FAA1F1B1FA81F10468EE
S315080017900425DBB29B0015FA03F334EA0303C9B246
S315080017A0890012FA01F11943016030BC7047C36819
S315080017B033EA1123090A91FAA1F1B1FA81F112FA71
S315080017C001F11943C1607047224909680843214954
S315080017D0086070471F49096831EA00001D4908601A
S315080017E0704710B501241C49884206D10420FFF72A
S315080017F0EBFF0420FFF7EEFF28E01849884206D1E0
S315080018000820FFF7E1FF0820FFF7E4FF1EE0144970
S31508001810884206D11020FFF7D7FF1020FFF7DAFF1E
S3150800182014E01049884206D12020FFF7CDFF20207A
S31508001830FFF7D0FF0AE00C49884206D14020FFF79F
S31508001840C3FF4020FFF7C6FF00E000242000C0B217
S3150800185010BD00000C10024000080140000C0140B9
S315080018600010014000140140001801402DE9F04124
S3150800187004000D0028680002060C96FAA6F0B0FAD5
S3150800188080F721E05FF0011039000839884050F0F0
S3150800189080686A6841462000FFF738FF2A69414692
S315080018A02000FFF784FF6868012802D068680928C5
S315080018B009D1AA6841462000FFF743FFEA68414676
S315080018C02000FFF759FF7F1C3000F84000280AD097
S315080018D03000F840C007F6D5082FD3D240F20110E1
S315080018E010FA07F8D5E70120BDE8F08180B5012098
S315080018F01549087000F01DF800F001F801BD80B523
S31508001900FEF78EFE012813D00F48007801280FD164
S31508001910FFF7C6F90D4909680D4A1268511811F5FD
S31508001920FA71884204D3002007490870FEF7ACFE16
S3150800193001BD80B504480078012803D1FFF7B0F946
S315080019400349086001BD00001E0D00200C0D002093
S31508001950080D0020002000080020000000400008B4
S315080019600020000000600008002000000080000839
S315080019700020000000A000080020000000C00008A9
S315080019800020000000E00008002000000000010818
S315080019900020000000200108002000000040010887
S315080019A000200000006001080020000000800108F7
S315080019B00020000000A001080020000000C0010867
S315080019C00020000000E0010800200000134800681D
S315080019D050F0010011490860114800681149084093
S315080019E00F4908600D4800680F4908400B49086010
S315080019F00A48006830F480200849086008480068EA
S31508001A0030F4FE00064908605FF41F0007490860C5
S31508001A105FF0006006490860704700000010024049
S31508001A20041002400000FFF8FFFFF6FE081002400F
S31508001A3008ED00E0433A5C576F726B5C736F66742F
S31508001A40776172655C4F70656E424C545C54617286
S31508001A506765745C44656D6F5C41524D434D335FF9
S31508001A6053544D333246315F4E75636C656F5F462E
S31508001A7031303352425F4941525C426F6F745C6D3C
S31508001A8061696E2E63000000433A5C576F726B5CA7
S31508001A90736F6674776172655C4F70656E424C54FD
S31508001AA05C5461726765745C536F757263655C41FB
S31508001AB0524D434D335F53544D333246315C756155
S31508001AC072742E630000000019E050F8041BCB075F
S31508001AD044BFA9F101035918121F0023042A41F82B
S31508001AE0043BF9D25FEA827C0B4604D54FF0000C22
S31508001AF0A1F800C09B1CD10744BF0021197050F8FB
S31508001B00042B002AE1D1704710B450F8041B79B1B0
S31508001B100268436802440830DC0744BFA9F101049F
S31508001B20E31852F8044B43F8044B091FF9D1ECE7C4
S31508001B3010BC704710B5074979441831064C7C44E7
S31508001B40163404E00A68081D114488470146A14274
S31508001B50F8D110BD08000000280000006DFFFFFF47
S31508001B601405000010080020000000009DFFFFFF7C
S31508001B700C000000840000000000002000000000A7
S31508001B8000F00BF8002801D0FFF7D4FF0020AFF3D0
S31508001B900080FFF749FC00F002F80120704700F0CA
S31508001BA001B800000746384600F002F8FBE70000D7
S31508001BB080B5AFF30080024A11001820ABBEFBE7E0
S31508001BC02600020002488546024880470248004728
S31508001BD010080020CD190008ED1B000800000000C1
S31508001BE0000000000102030406070809AFF300809D
S31508001BF0AFF30080FFF7C4FF1000000000A24A04FC
S31508001C000401000000000000010203044F70656E25
S31508001C10424C5400FFF7FEBFFFF7FEBFFFF7FEBFBB
S31508001C20FFF7FEBFFFF7FEBFFFF7FEBFFFF7FEBFDA
S31508001C30FFF7FEBFFFF7FEBFFFF7FEBFFFF7FEBFCA
S31508001C40FFF7FEBFFFF7FEBFFFF7FEBFFFF7FEBFBA
S31508001C50FFF7FEBFFFF7FEBFFFF7FEBFFFF7FEBFAA
S31508001C60FFF7FEBFFFF7FEBFFFF7FEBFFFF7FEBF9A
S31508001C70FFF7FEBFFFF7FEBFFFF7FEBFFFF7FEBF8A
S31508001C80FFF7FEBFFFF7FEBFFFF7FEBFFFF7FEBF7A
S31508001C90FFF7FEBFFFF7FEBFFFF7FEBFFFF7FEBF6A
S31508001CA0FFF7FEBFFFF7FEBFFFF7FEBFFFF7FEBF5A
S31508001CB0FFF7FEBFFFF7FEBFFFF7FEBFFFF7FEBF4A
S31508001CC0FFF7FEBFFFF7FEBFFFF7FEBFFFF7FEBF3A
S31508001CD0FFF7FEBFFFF7FEBFFFF7FEBFFFF7FEBF2A
S70508001BEDEA
